:100000000C9461000C947E000C947E000C947E0095
:100010000C947E000C947E000C947E000C947E0068
:100020000C947E000C947E000C947E000C947E0058
:100030000C947E000C947E000C947E000C947E0048
:100040000C94A4000C947E000C947E000C947E0012
:100050000C947E000C947E000C947E000C947E0028
:100060000C947E000C947E00000000002400270009
:100070002A0000000000250028002B0000000000DE
:1000800023002600290004040404040404040202DA
:100090000202020203030303030301020408102007
:1000A0004080010204081020010204081020000012
:1000B0000007000201000003040600000000000029
:1000C000000011241FBECFEFD8E0DEBFCDBF11E08E
:1000D000A0E0B1E0E6E9F3E002C005900D92A230A5
:1000E000B107D9F711E0A2E0B1E001C01D92AB3039
:1000F000B107E1F70E949D000C94C9010C94000027
:100100008091000161E00E947C0168EE73E080E074
:1001100090E00E94F8008091000160E00E947C0164
:1001200068EE73E080E090E00E94F800089580910E
:10013000000161E00E945C0108950E9422010E947A
:1001400097000E948000FDCF1F920F920FB60F9272
:1001500011242F933F934F935F936F937F938F93CC
:100160009F93AF93BF932091060130910701409177
:1001700008015091090170910A01DA01C901029642
:10018000A11DB11D672F6A5F6D3730F06D57DA0121
:10019000C9010396A11DB11D60930A018093060158
:1001A00090930701A0930801B09309018091020187
:1001B00090910301A0910401B09105010196A11D48
:1001C000B11D8093020190930301A0930401B093A9
:1001D0000501BF91AF919F918F917F916F915F9139
:1001E0004F913F912F910F900FBE0F901F90189538
:1001F000EF92FF920F931F937B018C018FB7F894BE
:100200004091060150910701609108017091090128
:100210008FBF2FB7F8948091060190910701A091AC
:100220000801B09109012FBF841B950BA60BB70BDA
:10023000E816F9060A071B0760F71F910F91FF9058
:10024000EF900895789484B5826084BD84B5816010
:1002500084BD85B5826085BD85B5816085BDEEE6CE
:10026000F0E0808181608083E1E8F0E0808182605D
:100270008083808181608083E0E8F0E0808181601C
:100280008083E1EBF0E0808184608083E0EBF0E04C
:10029000808181608083EAE7F0E0808184608083F0
:1002A000808182608083808181608083808180689A
:1002B00080831092C1000895282F30E0C90186562E
:1002C0009F4FFC0194912A573F4FF9018491882355
:1002D00091F0E82FF0E0EE0FFF1FE859FF4FA591D6
:1002E000B491662329F48C91909589238C93089579
:1002F0008C91892B8C930895482F50E0CA01825528
:100300009F4FFC012491CA0186569F4FFC01949196
:100310004A575F4FFA0134913323D1F1222331F14F
:10032000233021F4809180008F7705C0243031F490
:10033000809180008F7D8093800018C0213019F457
:1003400084B58F7704C0223021F484B58F7D84BDBD
:100350000DC0263021F48091B0008F7705C0273082
:1003600029F48091B0008F7D8093B000E32FF0E0FE
:10037000EE0FFF1FEE58FF4FA591B491662329F4AD
:100380008C91909589238C9308958C91892B8C93D3
:060390000895F894FFCF70
:02039600030062
:00000001FF
